:020000040000FA
:04000000E6EF01F036
:08000800E8CF05F0D8CF06F0A7
:10001000E0CF07F00001E9CF0DF0EACF08F0E1CF23
:1000200009F0E2CF0AF0D9CF0BF0DACF0CF0F3CF22
:1000300014F0F4CF15F0FACF16F000C00FF001C0A5
:1000400010F002C011F003C012F004C013F09DAA1A
:100050002DEF00F09EBA9CEF00F00FC000F010C032
:1000600001F011C002F012C003F013C004F00DC083
:10007000E9FF08C0EAFF09C0E1FF0AC0E2FF0BC0C8
:10008000D9FF0CC0DAFF14C0F3FF15C0F4FF16C08F
:10009000FAFF05C0E8FF07C0E0FF06C0D8FF100068
:1000A000F2CF0EF0F29EF76ABA0FF66E000EF7224C
:1000B0000900F5500EBEF28E1200496E6974696136
:1000C0006C697A696E6720506F727420420A0D0065
:1000D000F2CF0EF0F29EF76AEA0FF66E000EF722EC
:1000E0000900F5500EBEF28E1200436F6E6669670E
:1000F0007572696E672052462D3234470A0D000032
:10010000F2CF0EF0F29EF76A1A0FF66E010EF7228A
:100110000900F5500EBEF28E12004F4B210A0D0061
:100120009EAAFED7ABCF18F0AECF01F018A202D036
:10013000AB98AB880000000CF3DF01C028F028501A
:10014000120A01E025D0ECDF0150340802E0000E75
:1001500001D0010E2A6EE4DF0150560802E0000EC5
:1001600001D0010E2A142C6EDBDF0150780802E06A
:10017000000E01D0010E2C142E6ED2DF015090081B
:1001800002E0000E01D0010E2E14D8A4FF0000D012
:100190009E9A2DEF00F0EA6A200EE96EEF500FE014
:1001A000030E016E006A002EFED7012EFBD73C0E17
:1001B000006E002EFED700000000EF2EF1D7000CDD
:1001C000070E216E206A205007081DE3939A8A9A31
:1001D00021502106226E1FC000F02250016E04E063
:1001E000D8900032012EFCD700A003D093988A88C3
:1001F00002D093988A9800000000939A8A8A00009F
:100200000000202AE0D7000C93968A96939E8A9E3F
:10021000939A8A9A93988A98030E206EBCDF939ED5
:100220008A8E080E006E002EFED7100E1F6EC8DFDD
:10023000100E1F6EC5DF1F6AC3DF1F6AC1DF1F6A92
:10024000BFDF420E1F6EBCDF420E1F6EB9DF1F6A9A
:10025000B7DF1F6AB5DF1F6AB3DF420E1F6EB0DF64
:10026000420E1F6EADDF430E1F6EAADF6F0E1F6EB4
:10027000A7DF810E1F6EA4DF938893968A96939EC4
:100280008A9E939A8A9A55EF02F093968A96939E45
:100290008A8E080E006E002EFED793988A88939A55
:1002A0008A8A00000000939A8A9A00000000939EB8
:1002B0008A9E9388939A8A9A93968A8656EF02F03A
:1002C000236A070E246E226A225007082BE3939AB2
:1002D0008A9A00000000939A8A8A0000000093889E
:1002E00081A80FD024502406256E010E006E2550E3
:1002F000016E04E0D8900036012EFCD70050231286
:100300000FD024502406256E010E006E2550016E7C
:1003100004E0D8900036012EFCD70050FF0A2316C7
:10032000222AD2D723C001F0A5EF01F01F6A1F5087
:10033000010813E3036A1F50190F016E000E032218
:1003400001C020F003C021F0BBD721C0EAFF20C0CC
:10035000E9FF01C0EFFF1F2AEAD7939A8A9A939682
:100360008A866BEF02F0070E1F5E0CE3EA6A1F0E2F
:10037000E96ED890EF32EF5005E002D000000000A7
:10038000EF2EFCD7000C016A026A006A036A26504D
:1003900002E1255018E0100E276ED890233624363F
:1003A000003603362650035C02E12550005C07E36B
:1003B0002550005ED8A003062650035ED880013683
:1003C0000236272EEAD70000B3EF02F0F86AD09E7B
:1003D0000D8EEA6AE96AB8862A0EAF6E000EB06E1C
:1003E000260EAC6E900EAB6EC150C00B0F09C16EE5
:1003F000070EB46E186A7F0E1B6E1C6EC150C00BC8
:100400000F09C16EC290880ED56ECD6A000ECA6EFD
:100410007F0ECB6EB150480BB509B16EB70EB11659
:100420009484BD6ABD6AB1169482BA6ABA6A9D8A1A
:10043000C00EF2121F6A1F5033DE1F2A006E0050DA
:100440009EA8FED7AD6E130E1F5CF5E1030E206E65
:100450002E0E9EA8FED7AD6E202EFAD70A0E9EA8AD
:10046000FED7AD6E0D0E9EA8FED7AD6EF18EF29644
:100470001F6A1F502DDE1F2A006E00509EA8FED757
:10048000AD6E120E1F5CF5E1030E206E2E0E9EA8BF
:10049000FED7AD6E202EFAD70A0E9EA8FED7AD6EFF
:1004A0000D0E9EA8FED7AD6EAFD6EFD67F0E196E9D
:1004B0001A6E1F6A1F5024DE1F2A006E00509EA86D
:1004C000FED7AD6E050E1F5CF5E1B36AB26A938C80
:1004D00081AC07D02BD719C01BF01AC01CF0949820
:1004E0008B7893908A801E6A1E50030806E3D00E14
:1004F000006E002EFED71E2AF7D71E6A1E50030874
:1005000005E31BC01FF02FDF1E2AF8D793908A90B7
:1005100093928A821E6A1E50030806E3D00E006E74
:10052000002EFED71E2AF7D71E6A1E50030805E3C9
:100530001CC01FF018DF1E2AF8D793928A92B2507F
:10054000B3CF03F01F6E03C020F0D8901F34216E8C
:100550002034226E22C024F021C023F0020E266E29
:10056000710E256E10D701C01DF01D50130806E353
:10057000140ED8801D541F6E206E0DDEA6D703000A
:00000001FF
